:1000000009298030A100FE30A7200130A7207530DB
:10001000A7003030BE28A101A117AF00AF08031D13
:100020001328030114280130AF020310A20CA20C04
:10003000A20CC0302205403EAF07FE30A7202F089B
:10004000A728A101A117AF00FE30A7202F08A728DD
:10005000A401AA00AB01A01124080319A0150530C2
:10006000A3002730A900103041200330A900E83058
:100070004120A90164304120A9010A3041202A0809
:100080004828A8002B08A7002A08A600D220260886
:10009000A600A3030319A011240803195228230260
:1000A000031859282608031DA011A0195928303E0D
:1000B000A7280800AD0006118611831606118611C7
:1000C0000F30860583122D08A01884283E30A70023
:1000D0008030BE203330AC0098201330A700883029
:1000E000BE2098206430BD2098206430BD2022308E
:1000F000AC009820283083200C30832006308320E9
:10010000A0142D0884282014AC00201C92288611ED
:10011000033C031C972897200530A700DC30BE2045
:10012000031408002014FE3C0319A5288615201C82
:10013000201006150F3086052C08F03986040611AC
:10014000AC0E201898283230BD202D080429A11BA0
:100150005A2883178001840AFF3E031DAA28042918
:10016000A901A800FF30A807031CA907031C042944
:100170000330A700DF30BE20B228A701E83EA6006A
:10018000A709FC30031CC728A6070318C428A60724
:100190000000A70FC4282618CD28A61CD1280000CF
:1001A000D1280800AB01AA011030AC00270DAA0D20
:1001B000AB0D2808AA022908031C290FAB0203185B
:1001C000E8282808AA0729080318290FAB070310F5
:1001D000A60DA70DAC0BD628260804291030B000B8
:1001E000A701A601AD0CAC0C031CFC282808A6072F
:1001F00029080318290FA707A70CA60CAB0CAA0CFB
:10020000B00BF2282A080429831383120313000079
:100210000800A00107309F00E03083168500FF3002
:1002200086008113831285018601203084006030AE
:10023000AA20A03084005030AA2020308400303022
:10024000A920C830B020012077305A205A205A20E7
:100250002E305A2070305A2069305A2063305A208C
:1002600062305A2061305A2073305A2069305A2047
:1002700063305A202E305A206E305A206C305A206B
:100280000B30A900B830B120012044305A2043304F
:100290005A2046305A2031305A2036305A204E30BB
:1002A0005A204C305A2042305A2020305A205A20AE
:1002B00056305A202D305A2032305A200730A900AB
:1002C000D030B12001204C305A2044305A205230D6
:1002D0005A2020305A2061305A2066305A2072301D
:1002E0005A2065305A2067305A2065305A206C30C9
:1002F0005A2065305A206E305A2086188529851F6D
:1003000083290514842905107D29012053305A20A2
:1003100069305A2067305A206E305A2061305A2096
:100320005A206C305A2020305A207A305A206F30B0
:100330005A2065305A206B305A2065305A206E3072
:100340005A2036140512831605128312312AC3016E
:100350003C03A500C90149082502031CC029E3216B
:10036000B61CBE294308A6004908A200A601A20A9D
:100370000314A60DA20BB9292608C304C90FAB2983
:10038000B2014308B100B20CB10CB20CB10CB20C0A
:10039000B10CB20CB10C0F30B2053208AD0031080F
:1003A000AC00A9010A30A800EE20B1002B08B20071
:1003B000B4014308B3000F30B3050030B405310871
:1003C0003307C3000800BA01B9010618F829013043
:1003D000B020B90A0319BA0A0B303A02031CF729F4
:1003E000031DF629B9303902031CF7295F2CE529D2
:1003F0009B30B0200618B614061CB610361C112A05
:10040000440EB100B200F030B1050F30B205320831
:10041000A7003108A600A9013A30A800D220BD00EB
:10042000242A8030A1000130A2003D080D200230B6
:10043000A4004408292003013619013EB618013AE8
:1004400003193611031D3615C40A85140130A9009D
:10045000F430B1208510A901F030A8002808B1209F
:100460000800BB01C4013612361ACB2ABA01B90101
:10047000061C4B2AB90A0319BA0A0130B020AF3062
:100480003A02031C4A2A031D492AC9303902031CB7
:100490004A2A5F2C382ABA01B9010618872AB90AF4
:1004A0000319BA0A0A30B02036187B2A39080B3AE9
:1004B0003A04031D662A8030A1000130A2003D08E5
:1004C0000D2035305A2039305A207A2A3908193A05
:1004D0003A04031D6D2A85147A2A39084B3A3A04E6
:1004E000031D742A85107A2A3908FA3A3A04031D42
:1004F0007A2A5F2C862A11303A02031C862A031DB1
:10050000852A95303902031C862A5F2C4D2A4130FA
:100510003B02031C8C2A5F2CBB0A3A08031D942A59
:1005200065303902031C952A3616361CCA2A3B0E42
:10053000B100B200F030B1050F30B2053208A700AB
:100540003108A600A9014130A800D220BD008030AA
:10055000A1008030212053305A2069305A20673062
:100560005A206E305A2061305A205A206C305A205E
:1005700020305A2067305A2065305A2076305A2071
:100580006F305A206E305A2064305A2065305A201D
:100590006E305A20342A361CED2A012049305A2068
:1005A0006E305A2069305A2074305A2069305A20EF
:1005B00061305A206C305A2069305A2073305A20EA
:1005C00065305A2072305A2065305A206E305A20D9
:1005D0002E305A205A205A20572B0830BD000130A7
:1005E000A2003D080B20A101B61D052B3B304102A6
:1005F0000318FC2AC10A042BC10117304502031855
:10060000032BC50A042BC501092B4208C10046086B
:10061000C500051B192B4508031D112B0C30C70005
:10062000182B0D304502031C182B0C304502C70057
:100630001D2B4508C70020305A200A3047020318F6
:10064000232B20305A208030A100470828203A3040
:100650005A200230A400410829203A305A20303074
:100660005A205A20051B402B0C30450203183B2B07
:1006700061305A203D2B70305A200E30BD00422B85
:100680000F30BD00410803190130031D0301B500FF
:100690001E30410203190130031D03013504B5006A
:1006A00001308618030135040319572B372C361EE9
:1006B000352CE3210130C9000F3049020318632BA8
:1006C000E321C90F5C2B3611B611E321E321E321AD
:1006D000B61C6C2B05146D2B05101230C90014309C
:1006E00049020318762BE321C90F6F2BE321073052
:1006F000BC00A7214308C200E321361D802BB6159C
:100700000630BC00A7214308C600E321361D892B13
:10071000B6150630BC00A7214308BE000330BC005C
:10072000A7214308C8000530BC00A7214308C0002A
:100730000830BC00A7214308BF00E321361DA12BD0
:10074000B615361CA72BB619A62B36100120B619E4
:10075000342C8030A100803021203E082820203019
:100760005A2001304002031DBC2B6A305A206130F0
:100770005A206E305A20342C02304002031DC72B01
:1007800066305A2065305A2062305A20342C0330AB
:100790004002031DD22B6D305A2072305A20743023
:1007A0005A20342C04304002031DDD2B61305A20C6
:1007B00070305A2072305A20342C05304002031D0C
:1007C000E82B6D305A2065305A2069305A20342C7D
:1007D00006304002031DF32B6A305A2075305A2030
:1007E0006E305A20342C07304002031DFE2B6A3035
:1007F0005A2075305A206C305A20342C0830400270
:10080000031D092C61305A2075305A2067305A2058
:10081000342C09304002031D142C73305A206530EB
:100820005A2070305A20342C0A304002031D1F2CED
:100830006F305A206B305A2074305A20342C0B30D1
:100840004002031D2A2C6E305A206F305A20763019
:100850005A20342C0C304002031D342C64305A20B2
:1008600065305A2063305A20362C5F2C312A851F80
:100870003E2C0512831605128312402C8316051692
:1008800083129B30B020410803190130031D03017E
:10089000B50001308618030135040319502C0515E5
:1008A000851585140130A900F430B120051185119A
:1008B00085100130A9004A30B120C40A5A2B01200A
:1008C00047305A2065305A205A206E305A20203046
:1008D0005A2073305A2069305A2067305A206E30BF
:1008E0005A2061305A205A206C305A20203084001F
:1008F0006030AA20A03084005030AA20203084002C
:100900003030A9200618B616061CB61203010618C8
:10091000013EB61A013C031D932CB70A0319B80A0D
:100920000130B020862C0301B61A0130013A0319B8
:10093000B612031DB61603010618013EB61A013C95
:10094000031DA82CB70A0319B80A0130B0209B2C4C
:1009500003303802DE30031937020318762C3614C0
:02096000312A3A
:02400E00503F21
:00000001FF
